:100000000C94FC030C945C2E0C9434040C94340477
:100010000C9434040C9434040C9434040C94340480
:100020000C9434040C9434040C94A5250C94612590
:100030000C94A2260C9434040C9434040C943404D0
:100040000C9434040C9434040C9434040C94340450
:100050000C9434040C947E260C9434040C943404D4
:100060000C9434040C9434040C9434040C94340430
:100070000C9434040C9434040C9434040C94340420
:100080000C9434040C9434040C9434040C94340410
:100090000C9434040C9434040C9434040C94340400
:1000A0000C9434040C9434040C94340405010902B7
:1000B000A10185020901A1000509190129081500FE
:1000C0002501950875018102050109300931158165
:1000D000257F95027508810609381581257F9501D0
:1000E00075088106050C0A38021581257F95017572
:1000F000088106C0C005010980A101850319012AF4
:10010000B700150126B700950175108100C0050CD8
:100110000901A101850419012AA002150126A002E6
:10012000950175108100C00660FF0961A101096297
:10013000150026FF00952075088102096315002629
:10014000FF00952075089102C005010906A101056F
:100150000719E029E7150025019508750181029529
:1001600001750881010507190029FF150026FF0008
:100170009506750881000508190129059505750181
:100180009102950175039101C0000000000000007C
:10019000000000000000000000000000000000005F
:1001A000000000000000000000000000007E0F00C2
:1001B000D4FFFFFFC700000078000000000000002F
:1001C000002A2B28000000000000000000000000B2
:1001D0000000000029000000002C1E3420212224F1
:1001E000342627252E362D3738271E1F202122237F
:1001F0002425263333362E37381F04050607080911
:100200000A0B0C0D0E0F10111213141516171819D6
:100210001A1B1C1D2F3130232D3504050607080934
:100220000A0B0C0D0E0F10111213141516171819B6
:100230001A1B1C1D2F3130354C1E0F0500047F3F4B
:100240001F643214643214783C1E1E140A05000127
:100250000101010101010101020202020202020286
:100260000203030303030303030404040404040458
:10027000050505050506060606060707070707081C
:10028000080808090909090A0A0A0B0B0B0C0C0CCF
:100290000D0D0D0E0E0E0F0F0F1010111111121269
:1002A00013131414151516161717181819191A1AE6
:1002B0001B1B1C1D1D1E1E1F202021222223242447
:1002C000252626272829292A2B2C2D2D2E2F303183
:1002D0003232333435363738393A3B3C3D3E3F4095
:1002E0004142434445464748494A4C4D4E4F505180
:1002F0005354555658595A5B5D5E5F61626465663A
:1003000068696B6C6D6F7072737577787A7B7D7EC0
:100310008082838587888A8C8E8F91939596989A10
:100320009C9EA0A2A3A5A7A9ABADAFB1B3B5B7BA28
:10033000BCBEC0C2C4C6C9CBCDCFD1D4D6D8DBDDFC
:10034000DFE2E4E7E9EBEEF0F3F5F8FAFDFFFFAAF0
:100350007F55400102030C0D0E0F00070605040B2C
:100360000A09082223252628292A2C2D2F3032334A
:100370003536383A3B3D3E4042434547494A4C4E6C
:100380005051535557595A5C5E6062646668696B98
:100390006D6F71737577797B7D7F81838587898A9E
:1003A0008C8E90929496989A9C9E9FA1A3A5A7A8A4
:1003B000AAACAEAFB1B3B4B6B8B9BBBCBEBFC1C2D4
:1003C000C3C5C6C7C9CACBCCCDCED0D1D2D2D3D467
:1003D000D5D6D7D7D8D9D9DADADBDBDBDCDCDCDC85
:1003E000DCDDDDDDDDDCDCDCDCDCDBDBDBDADAD953
:1003F000D9D8D7D7D6D5D4D3D2D2D1D0CECDCCCBD5
:10040000CAC9C7C6C5C3C2C1BFBEBCBBB9B8B6B4F2
:10041000B3B1AFAEACAAA8A7A5A3A19F9E9C9A9882
:10042000969492908E8C8A89878583817F7D7B7953
:10043000777573716F6D6B6968666462605E5C5A34
:100440005957555351504E4C4A4947454342403EF7
:100450003D3B3A3836353332302F2D2C2A29282689
:100460002523223A003B00167C1E001F002000219D
:1004700000220023003C003D002B0014001A00085D
:10048000001500170000003E003F00390004001670
:1004900000070009000A00000040004100E100647C
:1004A000001D001B0006001900050042004300E08B
:1004B00000E200E30021522C002C00000024002563
:1004C00000260027002D002E004C002A004A001CA8
:1004D0000018000C00120013002F00300031004DF6
:1004E000000B000D000E000F003300340032002816
:1004F000004B00110010003600370038000000E506
:100500000052004E0021522C00E600E400E70000FB
:1005100000500051004F0001000100167C3A003BE2
:10052000003C003D003E003F00010001002078211A
:1005300078010052000100010000000100010001EB
:10054000000100500051004F0001000000010001B7
:100550000001000100010001000100010001000193
:10056000000100350201000100010001000100004E
:10057000004000410042004300440045004C002A76
:100580000001000100010001000100010001000163
:100590000001000100010001000100010001000153
:1005A0000001000100010001000100010001000143
:1005B0000000000100010001000100010001000134
:1005C0000001000000010001000100010001000124
:1005D0000001000100010001000100010001000113
:1005E0000001000100010001000100010000000104
:1005F00000010001000100010001000100010000F4
:1006000000010001000100010001000100010001E2
:1006100000010001000100010001000100010001D2
:1006200000010000000100010001000100010001C3
:1006300000010001000100010001000100010001B2
:1006400000010001000100010001000100010001A2
:100650000001000100010001000100010001000192
:100660000001000100000001000100010001000183
:100670000001000100010000000100010001000173
:100680000001000100010001000100010001000162
:100690000001000100010001000100010001000152
:1006A0000000000100010001000100010001000143
:1006B0000001000000010001000100010001000133
:1006C0000001000100010001000100010001000122
:1006D0000001000100010000000100010001000113
:1006E0000001000100010001000100010001000102
:1006F00000010001000100010001000100010001F2
:1007000000010001000100010001000100010001E1
:1007100000010001000100010000000100010001D2
:1007200000010001000100010001000000010001C2
:100730000001004E004B00A900AA0021782278ABEE
:1007400000AC00237824782578267829782A782721
:1007500078287809025B00030100A0FA0904000070
:1007600001030101000921110100012240000705D8
:1007700081030800010904010002030000000921AF
:100780001101000122220007058203200001070554
:1007900003032000010904020001030000000921F5
:1007A00011010001227B00070584032000011201D2
:1007B00000020000000810CB575310050102000191
:1007C00022035100750065006600720065006E002E
:1007D0006300790020005200650076002E002000A2
:1007E000350000000E034B006500650062006900E3
:1007F0006F0000000403090411241FBECFEFDAE0EC
:10080000DEBFCDBF04B603FE18C08091CE03909129
:10081000CF03A091D003B091D1038730904BA74074
:10082000B04B59F41092CE031092CF031092D00324
:100830001092D103E0E0F8E3099523E0A4EFB1E0E2
:1008400001C01D92AE3CB207E1F711E0A0E0B1E0BB
:10085000E8E2F3E602C005900D92A43FB107D9F794
:100860000E94C9260C9429310C940000482F209135
:10087000CA039091910357E0291302C080E00895C4
:1008800030E0529FF001539FF00D1124EE56FC4FC3
:100890008181681306C08081481303C0858181115E
:1008A000EECF2F5F3F4F2770E7CFE8EDF0E080817C
:1008B0008E7F80831092E2001092DA001092E100A5
:1008C000A0EEB0E08C9181608C9380818F778083E3
:1008D00019BCA7EDB0E08C918E7F8C9380818F7EC8
:1008E000808310927A0308952091E4003091E5000E
:1008F00095E6A9012091EC00822F817020FF06C0AF
:100900008091E80080FF06C080E008952091E80013
:1009100022FD1AC080918703882389F0853089F0F1
:100920008091EB0085FD0FC02091E4003091E5003F
:1009300042175307F9F29150E1F684E0089582E0FE
:10094000089583E0089581E008958091890387FFE9
:1009500013C08091E80082FF06C08091E8008B7789
:100960008093E80004C0809187038111F2CF08953D
:10097000809187038823D9F38091E80080FFF8CF26
:100980008091E8008E77ECCF982F9093E900242F88
:10099000762F50E0891731F07091EC002091ED0036
:1009A0005091F00021FD07C09F5F973071F7809351
:1009B000E90081E008953091EB003E7F3093EB0039
:1009C0003091ED003D7F3093ED003091EB003160D0
:1009D0003093EB007093EC002093ED005093F00007
:1009E0002091EE0027FDE0CF80E00895B0E0A0E088
:1009F000ECEFF4E00C94822FC8EDD0E088818F7E7C
:100A00008883E7EDF0E080818160808384E082BFAD
:100A100081E080937A0388818E7F888302EE10E0E4
:100A2000F80110821092DA0081EEC82ED12CF60166
:100A3000108288818F778883888180688883888105
:100A40008F7D888319BC10928703109288031092BF
:100A500086031092850390EEE92EF12CF701808138
:100A60008B7F808388818160888342E060E080E0C2
:100A70000E94C404F60180818E7F8083F80180810A
:100A800081608083808188608083F70180818E7F90
:100A90008083888180618883CDB7DEB7E8E00C94DD
:100AA0009E2FFC0180918F039091900386179707EA
:100AB000A0F06115710529F49091E8009E7790935C
:100AC000E80090E06115710551F4911108C0809122
:100AD000E80082FF34C080E00895BC01F2CF80912D
:100AE00087038823C1F18530C1F18091E80083FD3F
:100AF00030C08091E80082FDEACF8091E80080FF5D
:100B0000E1CF8091F3002091F200382F611571053B
:100B100019F02830310558F091E02830310509F0FE
:100B200090E02091E8002E772093E800CBCF8191D0
:100B30008093F100615071092F5F3F4FE7CF8091A3
:100B40008703882341F0853041F08091E80083FFDE
:100B5000BECF81E0089582E0089583E008958091FA
:100B60007C0308959C014FB7F8948091760390918F
:100B70007703A0917803B09179034FBF821B930B49
:100B800008952FB7F8946091760370917703809160
:100B90007803909179032FBF08952FB7F89480912F
:100BA000760390917703A0917803B09179032FBFDA
:100BB0000895A3E0B0E0EFEDF5E00C94882F2091CC
:100BC00073033091740328173907A1F090937403CD
:100BD00080937303E0917103F0917203309751F0A9
:100BE00024E029839B838A830680F781E02DCE0150
:100BF000019609952396E2E00C94A42FA3E0B0E0BF
:100C0000E4E0F6E00C94882F20916F03309170039C
:100C100028173907A1F09093700380936F03E09138
:100C20007103F0917203309751F023E029839B8385
:100C30008A830680F781E02DCE01019609952396DF
:100C4000E2E00C94A42FFC01680F791F8FEF91E371
:100C50002191822728E030E087FF09C0880F89278B
:100C600021503109C9F7E617F70791F70895880F62
:100C7000F7CFFA01811101C0FB010995089508958C
:100C8000E4EEF2E011828281846082830895809193
:100C90006A03982F9E7F29F48170826080936A0393
:100CA00008958635E8F381708465F8CFAF92BF92DE
:100CB000DF92EF92FF920F931F93CF93DF93082F52
:100CC000162FE901E42FF0E0E25BFD4F611110C047
:100CD000E4915E2F4E2F4983E8835A83DF91CF91B1
:100CE0001F910F91FF90EF90DF90BF90AF9008950C
:100CF000E62EF12C4491D42EE42FF0E026E0829FE2
:100D0000C00111242FEF30E0B9010E94BB2F802FCA
:100D100090E0880F991F55E5569FD001579FB00D61
:100D200011248A1B9B0B982F990F890F5901AE181C
:100D3000BF08AE9ED001AF9EB00DBE9EB00D112477
:100D40005B2F189F80011124012F11275901A01A30
:100D5000B10AAE9E8001AF9E100DBE9E100D1124F3
:100D60005901A81AB108AE9CC001AF9C900DBE9C61
:100D7000900D1124892F9927281B390B2E9FC00114
:100D80002F9F900D3E9F900D1124E92F6230710529
:100D9000A1F050F46115710509F49DCF6130710522
:100DA00081F0EB2F512F97CF6430710569F080F0FF
:100DB0006630710509F48FCFF4CFE42F4B2F592FF4
:100DC0008ACFE42F412F87CFEB2F542F492F83CF8A
:100DD0004B2F5D2DE12F7FCF0E94CD059C0190917F
:100DE000DA028091DB02982B21F03093D702209316
:100DF000D6029091DC028091DD02982B21F0309395
:100E0000D5022093D402E0917103F09172033097E0
:100E100049F082E08093D8020480F581E02D88EDCE
:100E200092E0099508958091D30280FD16C081FD5E
:100E300016C082FD16C08091D2028823A1F08832AC
:100E400080F428E0829FC001112468E270E00E94D3
:100E5000CF2F862F672B39F0089582E0089584E024
:100E6000089588E0089581E008958091D30280FD7F
:100E700014C081FD14C082FD16C08091D102882368
:100E800081F08E3180F420E5829FC00111246EE153
:100E900070E00E94CF2F862F089584E1089588E2A4
:100EA000089588E0089580E5089580E00895F89415
:100EB000E82FE295EF70F0E031A1282F2F7081E04C
:100EC00090E001C0880F2A95EAF7982F9095932318
:100ED00091A392A1892B82A378940895909199026D
:100EE00092FF06C0282F28712830F9F4877F84608C
:100EF00093FF06C0282F28712831F1F4877E846182
:100F000020919A0220FF06C0382F38713830D9F46A
:100F1000877F816021FF06C0282F28712831D1F4F6
:100F2000877E816194FD877E0895282F2471243067
:100F3000F9F68B7F8860DCCF282F2471243101F7EC
:100F40008B7E8861DDCF382F3171313019F78E7F7C
:100F50008860E0CF282F2171213121F78E7E8861B2
:100F6000E1CF82389105B9F1B0F48133910509F4EC
:100F70007DC048F48932910509F46DC08A3291052B
:100F800009F47BC008958533910509F45FC0893366
:100F9000910509F10895833E9105D9F138F4803E19
:100FA000910529F1823E910579F10895863E9105DA
:100FB000D9F1873E910509F43EC0843E910541F583
:100FC00020919A0221FF24C08091990284FD19C0CA
:100FD00087EE90E0089520919902237009F05AC09D
:100FE00020919A0223FF14C089E290E00895209195
:100FF000990220FD38C030919A0230FF09C024FFC9
:1010000043C090E080E008952091990222FDF7CF3F
:1010100008952091990222FD3AC030919A0230FD44
:1010200039C024FFF5CFEDCF2091990223FFF0CFF7
:1010300024FDE7CFCDCF2091990223FD2EC0309122
:101040009A0231FFEECF84EE90E00895209199024C
:1010500025FFDECFC9CF2091990225FD21C0209127
:101060009A0223FFD5CF89E390E0D2CF2091990255
:1010700026FFCECF8AE290E008952091990226FFC4
:10108000C7CF81E390E0089583EE90E0089582EE6B
:1010900090E0089580EE90E0089586EE90E0089547
:1010A00085E390E008951F93CF93DF930E94B107EB
:1010B000EC01C11580E5D807F0F5C11580E4D8072B
:1010C00008F09CC0C03ED10520F5CD3CD10508F00C
:1010D00082C0C83AD10578F4C53AD10508F073C08A
:1010E000C130D10519F1209709F1C430D105F0F4D0
:1010F000D0E0C0E01BC0C33CD105D0F7C85AD0E057
:10110000CC0FDD1FCE58DE4F0990D881C02DD4649E
:101110000DC0C11580E2D80708F0D1C0C11581E02B
:10112000D80708F05AC0C83ED10510F7CE01DF91AC
:10113000CF911F910895C03682E5D80718F5C034C5
:1011400082E5D80708F06BC0C03282E5D80708F006
:101150005FC0C11582E5D80708F497C02C2F2695EB
:10116000269580E2289F900111248C2F8370C1E086
:10117000D0E002C0CC0FDD1F8A95E2F7C22BD32B43
:10118000DD68D4CFC03A82E5D80760F4C03882E584
:10119000D80708F459C0CF71D0E0DC2FCC27C46F3A
:1011A000D06AC4CFC03C82E5D80708F462C0C03E14
:1011B00082E5D80708F09CCFDC2FCC27CC27DF7145
:1011C000C06FD06AB3CFC55AD0E0C159DE4FC881D5
:1011D000D0E0D064ABCFD065A9CF8D2F0E946E0731
:1011E000182FCE0199270E94B107C12FD0E0DC2F24
:1011F000CC27CC27DF71C82BD92B98CFCE019927CC
:101200000E94B107CC27DF70C82BD92BD06A8ECFB4
:10121000CF71D0E0DC2FCC27C16FD06A87CF2C2FC5
:1012200026952695277080E2289F900111248C2F07
:101230008370C1E0D0E002C0CC0FDD1F8A95E2F7D9
:10124000C22BD32BDC6872CF2C2F269526952770C6
:1012500080E2289F900111248C2F8370C1E0D0E0A0
:1012600002C0CC0FDD1F8A95E2F7C22BD32BDA68C0
:101270005DCF8C2F8F710E946E07C82FD0E0DC2FBE
:10128000CC27CC27DF71D06251CF8C2F8F710E9479
:101290006E0755E0D695C7955A95E1F7CF70D0E027
:1012A000DC2FCC27282F30E084FF05C044E0220F3C
:1012B000331F4A95E1F7C22BD32BD06937CF8D2F3F
:1012C0008F710E946E07182FCE0199270E94B107D7
:1012D000C12FD0E0DC2FCC27CC27DF71C82BD92B36
:1012E000D2CF809590913902982390933902089536
:1012F000E8EFF1E09191891303C0DF0111971C928F
:1013000091E0EE3FF907B1F70895A8EFB1E0EFEFF4
:1013100090E02D91821751F0EF3F19F4211101C097
:10132000E92F9F5F9630A9F7EF3F09F408950E2E3D
:10133000000CFF0BEA50FE4F828308958091CA0390
:1013400090919103981301C008958F5F8770FACF31
:10135000A82FA77023E0969587952A95E1F7FC01C1
:10136000EE0FFF1FE80FF91FE60FF71F50E040E0F8
:1013700080E0219130E00A2E02C0369527950A942C
:10138000E2F721703327042E01C0220F0A94EAF7F6
:10139000822B4F5F5F4F4330510559F70895292F36
:1013A0009A3068F4893090F490E063E072E039E0BC
:1013B000239F800D911D11240E94A80908952C5F80
:1013C000223020F460E072E090E0F6CF80E00895F3
:1013D000262F277091E001C0990F2A95EAF723E0A4
:1013E000769567952A95E1F7FB01EE0FFF1FE60F53
:1013F000F71FE40FF51F50E040E0682F70E0819187
:10140000DF0111979B01042E02C0369527950A949F
:10141000E2F7217021952827292328272C934F5F55
:101420005F4F4330510559F70895282F862F9A3082
:1014300070F4293058F4622F70E029E0929F600D1B
:10144000711D112443E052E00E94E80908959C5F59
:101450009230E0F7622F70E040E052E0F5CF8093E9
:10146000980208959091980221E030E0F90101C0BE
:10147000EE0F8A95EAF7D90102C0AA0FBB1F6A9541
:10148000E2F7EA2B01C0220F4A95EAF7892F8E2353
:10149000E81305C0292B822F0E942F0A089520955A
:1014A0002923F9CF21E030E001C0220F8A95EAF725
:1014B00020958091980282230E942F0A089590918E
:1014C0002E028095892380932E02282F277069F49D
:1014D000891759F090919A0292FF07C086958695D8
:1014E00086950E94520A10922E02089521E030E063
:1014F00001C0220F8A95EAF780919802822B0E9400
:101500002F0A089580933A020895662309F45DC076
:101510008D3C41F40E94350781958093DB020E9447
:10152000EC0608958E3C19F40E943507F6CF8F3CE7
:1015300031F40E94350781958093DA02F0CF803D27
:1015400019F40E943507F8CF893D29F40E9413074A
:101550008093DC02E4CF8A3D21F40E941307819539
:10156000F7CF8B3D31F40E94130781958093DD0204
:10157000D6CF8C3D19F40E941307F8CF9FE2980F45
:10158000983070F4815D990B21E030E001C0220FAA
:101590008A95EAF78091D902822B8093D902BFCF36
:1015A0008D3D31F48091D30281608093D302B7CF17
:1015B0008E3D21F48091D3028260F7CF8F3D09F0F8
:1015C000AECF8091D3028460F0CF4091DA028D3C9F
:1015D00059F48091DB0287FF0DC01092DB024111AC
:1015E0000BC01092D10208C08E3C81F48091DB02C6
:1015F00018169CF3442381F08091DC029091DD0267
:10160000892B09F08CCF1092D20289CF8F3C49F4FC
:1016100047FFF0CF1092DA028091DB028111ECCF0C
:10162000E0CF803D19F41416ACF3E4CF9091DC02C6
:10163000893D29F41916F4F61092DC02DBCF8A3DBD
:1016400019F497FFD7CFF8CF9091DD028B3D29F4A5
:1016500097FFD0CF1092DD02CDCF8C3D19F4191633
:10166000CCF3C8CF9FE2980F983090F4815D990B2E
:1016700021E030E0B90102C0660F771F8A95E2F7DA
:10168000CB0180959091D90289238093D902B2CF62
:101690008D3D31F48091D3028E7F8093D302AACF07
:1016A0008E3D21F48091D3028D7FF7CF8F3D09F0DD
:1016B000A1CF8091D3028B7FF0CF0F931F93CF9355
:1016C000DF938B01EA0190918703943061F5809359
:1016D000E9008FEF9091E800815095FD06C095EDEF
:1016E0009A95F1F700008111F5CF8091E80085FF10
:1016F0001AC00E947404811111C08091E80085FD18
:1017000006C08091E8008E778093E800F2CFF80160
:1017100081918F018093F100219779F78091E80002
:101720008E778093E800DF91CF911F910F910895FC
:1017300043E050E0BC0184E00E945D0B089546E068
:1017400050E0BC0184E00E945D0B0895CF93DF93CD
:10175000EC0148E050E0BC0181E00E945D0B88E0B4
:10176000FE01ADE7B3E001900D928A95E1F7DF91BC
:10177000CF91089581E08093E00080E28093D800CB
:101780001092C9008FE19EE40197F1F700C00000BC
:1017900087E090EBDC018093CE039093CF03A0937E
:1017A000D003B093D10388E19CE00FB6F894A895DC
:1017B000809360000FBE90936000FFCFCF92DF92C6
:1017C000EF920F931F93CF93DF93CDB7DEB7E097E0
:1017D0000FB6F894DEBF0FBECDBF60915C01809163
:1017E0006A0380FF4BC0E3E5F3E09E012F5F3F4FAC
:1017F0008E010F5C1F4FC901A4914A2F50E0DA01FE
:10180000AA0FBB1FA40FB51FA651BD4FCD90DD90F1
:10181000EC90D901CD92DD92ED929D013196A01709
:10182000B10751F720915B0143E0249F800D911D8A
:1018300011246E9A2EB12F7B3EB130645FB7F894BD
:10184000FC01649FE00DF11D1124BF01861797076D
:1018500041F55FBFEFE5F4E03197F1F700C000001C
:10186000E0960FB6F894DEBF0FBECDBFDF91CF91EB
:101870001F910F91EF90DF90CF90089580915D01BF
:1018800090915E0123E0829FF0011124E651FD4F0B
:10189000891708F0A8CF1182108212828F5F3396C9
:1018A000F7CFDC014D91CD01E8E03EB9000000C06A
:1018B00047FF2EB9440F000000C000C000C02EB981
:1018C00000C0EA9591F7C2CF0F931F93CF93DF9398
:1018D000EC0110E000E090915F019017110609F013
:1018E0006CF40E94DE0B8C8190E001968170992748
:1018F0008C83DF91CF911F910F91089520915D010D
:10190000A801420F511D9A01220F331F240F351FCA
:1019100026513D4F4C8160916C0380916B039695ED
:101920009017110651F04CF0442349F040916D039B
:101930000E9456060F5F1F4FCECF4423B9F340E0FD
:10194000F7CFB0E0A0E0E7EAFCE00C947E2FEC01DA
:101950004C81042F10E09801D8010E941A319B019C
:10196000AC010E94E5304B015C01E0E2F0E0E01BDD
:10197000F10BA5E5B0E0AC019B010E94E5306B01E5
:101980007C019F01DF010E94F02F9B01AC010E94AE
:10199000F0309B01AC01280D391D4A1D5B1DC701AC
:1019A000B6010E94F830F22E822F90E039E23F1506
:1019B00020F143E0249F9001112435952795122FA3
:1019C000109500E085E5E82EEF1880915F0108177B
:1019D00018F10E94DE0B9C8181E0992319F090326E
:1019E00019F48FEF80935A0180915A01890F8C83EB
:1019F000CDB7DEB7ECE00C949A2F25E530E0B901C5
:101A0000681B790B9B01220F331F260F371F37FFEF
:101A1000D4CF2F5F3F4FD1CF8E2D01FD8F2D209141
:101A20005D01622F600F7727771F9B01220F331F05
:101A3000260F371F26513D4F412F60916C030E94A6
:101A400056060F5FC2CFEF92FF920F931F93CF9373
:101A5000DF93EC018C81811109C081E08C831092AD
:101A6000E80292E0909359018093580180915D01C2
:101A700090915E0123E0829FF0011124E651FD4F19
:101A8000891758F110E003E060915F01161758F1D3
:101A90000E94DE0B809158012091E802280F2093CC
:101AA000E80290915901980F90935901191654F436
:101AB000022E000C330B40915F014150550B24174F
:101AC000350734F0819580935801813009F41C82E8
:101AD000CDB7DEB7E6E00C94A02F118210821282FF
:101AE0008F5F3396CDCFE12EF12C70E0C7010E94BD
:101AF000CF2F20915D01820F482F50E02091E80206
:101B0000022E000C330BE216F306BCF020915901B3
:101B1000022E000C330B2E153F057CF0809F9001A8
:101B2000112426513D4F40916D0360916C038091CB
:101B30006B030E9456061F5FA7CFFA01EE0FFF1F2F
:101B4000E40FF51FE651FD4F118210821282F3CF90
:101B5000B0E0A0E0EEEAFDE00C947F2FEC018A817A
:101B6000BB24BA9480FD02C0BB24B394A0905F0153
:101B70008C81811109C081E0B8121EC08FEF8A0DDF
:101B80008093E70281E08C83F12CE12CEA14B8F019
:101B90000E94DE0B8091E70291E0B91254C08111DE
:101BA0004DC080915F0181508093E7021C82CDB7C8
:101BB000DEB7EBE00C949B2F1092E702E3CF00918D
:101BC0005D010E0D1F2D111DC801880F991F080FF3
:101BD000191F06511D4FF80111821082128234E044
:101BE000C32ED12C912C8091E702890D813114F103
:101BF0008F70082E000C990B8E159F0591F4809123
:101C00006D038C9DA0018D9D500D11245595479518
:101C100055954795980160916C0380916B030E94E4
:101C200056069B0CF1E0CF1AD108E9F68FEFE81ABF
:101C3000F80AACCF87FFDDCF8A0DDBCF81508093D0
:101C4000E702BC82B4CF90E0019660915F0170E042
:101C50000E94CF2F8093E7028C83A9CFEF92FF924F
:101C60001F93CF93DF93EC0110E0EE24EA94F12C64
:101C700060915F01161770F00E94DE0B9A818C81D3
:101C800090FF27C08F5F8C83DF91CF911F91FF90D2
:101C9000EF90089520915D01422F410F5527551F68
:101CA000CA019A01220F331F280F391F26513D4FB9
:101CB00070E0C7010E94CF2F962F8C8140916D0359
:101CC00060916C03199F800D11240E9456061F5FBE
:101CD000CFCF8150D8CF90916A0390FF0EC09091E2
:101CE0005D0120915E0133E0939FF0011124E651E4
:101CF000FD4F921718F00E94DE0B089581836083D8
:101D000042839F5F3396F5CFA3E0B0E0EAE8FEE0C0
:101D10000C94862F8C018091E90281110AC09E01EA
:101D20002F5F3F4F4FEF6FEF0E9456068A818093DF
:101D3000E902F8016481613069F08091E90240E0D4
:101D4000662361F040E0623011F44091E90280E0E6
:101D500060E004C06091E90240E080E00E946B0E08
:101D6000F801848190E0019663E070E00E94CF2F3B
:101D700084832396E4E00C94A22FA3E0B0E0E3EC8C
:101D8000FEE00C94882F90916A0390FF0AC09E0198
:101D90002F5F3F4F0E9456064B8169818A810E94C6
:101DA0006B0E2396E2E00C94A42FCF93DF93EC010B
:101DB000EAE6F3E0438162818C810E94BD0E8C8152
:101DC0008F5F8C83DF91CF910895CF93DF93EC01E8
:101DD000EC81F0E0ED59FC4F4491EAE6F3E06281DA
:101DE00081810E94BD0E8C818F5F8C83DF91CF91AA
:101DF0000895EAE6F3E080818E7F80830E944006AA
:101E0000E4EEF2E08281816082830E94DE0B08951D
:101E1000B0E0A0E0EEE0FFE00C94802F7C015B01DD
:101E20006A0180917B0201E010E08A3010F40AE040
:101E300010E0C1E0D0E0B501C701F60109958111BC
:101E400004C021960C171D072CF4CDB7DEB7EAE0CD
:101E50000C949C2FCC9F9001CD9F300D300D112400
:101E600090E080E045E34A95F1F700000196821783
:101E70009307C1F7E0CF80914702811110C0809194
:101E8000D80080618093D8008AE18A95F1F700C07C
:101E90008091D90080FF0AC081E08093470281E0F1
:101EA00090914702913009F080E0089582E080939C
:101EB00047020E94550410928703F1CF0E943B0F06
:101EC000882359F0E0917103F0917203309729F063
:101ED0000190F081E02D0995089580E008950F9319
:101EE0001F930E943B0F882329F00E94C1051F9178
:101EF0000F9108950E94C10500917C0210917D020E
:101F000020917E0230917F02600F711F821F931F0C
:101F1000EECF0E946F0F08950E943B0F882319F0A7
:101F20000E94CD0508950E946F0FCB010895CF93B5
:101F3000DF93C6E1D3E060E0CE010E9492302196AB
:101F4000C11584E0D807B9F7DF91CF9108950F93B9
:101F50001F93CF93DF93142F022F843020F562302C
:101F600010F598E0899FE001112484E0689FB0019A
:101F70001124C60FD71FCA50DD4F82E090E04423E2
:101F800011F090E080E0632F8C0F9D1F0E94923033
:101F900083E090E0112311F081E090E0602F8C0F3E
:101FA0009D1F0E949230DF91CF911F910F91089554
:101FB0001F93CF93DF93122F8430E0F46A30D0F474
:101FC0004930C0F4C42FD0E0CC0FDD1F92E1699FEF
:101FD000C00DD11D112494EB899FC00DD11D11247A
:101FE000632FCE0186960E949230612FCE01879694
:101FF0000E949230DF91CF911F910895B0E0A0E050
:10200000E4E0F0E10C947E2F83E3E82E87E0F82EE5
:1020100003E614E0C0E05801D0E015C0F4012591BA
:1020200034914D2D6D2F8C2F0E94D80F82E0880E99
:10203000911CD39489E0D812F1CF82E1A80EB11C93
:10204000DF5FDA3019F04501D12CE8CF6701D0E02D
:10205000F6012591349141E06D2F8C2F0E94A70F3E
:10206000F60132962591349140E06D2F8C2F0E941D
:10207000A70F84E0C80ED11CD13071F488E0E80EBF
:10208000F11CCF5F0C541F4FC43009F0C4CFCDB743
:10209000DEB7ECE00C949A2FD1E0DACFCF93C82FC3
:1020A0006FEF811162E282E290E00E9492306FEF66
:1020B000C11163E083E290E00E9492306FEFC111A2
:1020C00060E184E290E00E949230CF91089580E038
:1020D0000E944E1060E085E290E00E9492300E94E3
:1020E000FE0F0E94970F81E00E944E100895FF920C
:1020F0000F931F93CF93DF93F42E843070F56230EB
:1021000060F528E0829F8001112434E0639FB001D4
:102110001124060F171F0A501D4F82E090E0442340
:1021200011F090E080E0800F911F0E947E30C82F58
:10213000D0E0DC2FCC2783E090E0FF2011F081E09D
:1021400090E0800F911F0E947E309E01282BC901D4
:10215000CDB7DEB7E5E00C94A12F90E080E0F8CF9A
:102160000F931F93CF93DF93843030F56A3020F5BF
:10217000493010F5C42FD0E0CC0FDD1F22E1629F63
:10218000C00DD11D112434EB839FC00DD11D11242E
:10219000CE0186960E947E30082F10E0102F002777
:1021A000CE0187960E947E309801282BC901DF91CD
:1021B000CF911F910F91089590E080E0F8CF7A3091
:1021C00048F4693070F4843060F4462F672F0E9421
:1021D000B01008957D3F41F4623018F441E084303E
:1021E00050F090E080E008957C3FD9F76230C8F766
:1021F0008430B8F740E00E9477100895CF92DF92C4
:10220000FF920F931F93CF93DF936C01009198027D
:1022100080913A02082BC3E0D0E010E0FC2EC80108
:102220000C2E02C0959587950A94E2F780FD0CC0AC
:102230002197A0F7F12C8F2DDF91CF911F910F9156
:10224000FF90DF90CF900895B6018C2F0E94DF1091
:102250000E945308019761F3EECFCF93DF93EC0117
:102260000E94FE10BE010E94DF100E945308DF9101
:10227000CF910895FC0124812223C1F080819181B6
:102280000E942D1192959F70963091F058F4925FB4
:102290009F70923058F4803F19F030F4883E30F44B
:1022A00081E008959A5FF4CF843FD1F380E00895F0
:1022B000883EB0F3813FD1F7F3CF82E290E00E94F5
:1022C0007E30823289F483E290E00E947E30833057
:1022D00059F484E290E00E947E3091E0803109F070
:1022E00090E0892F8170089580E0FCCFB0E0A0E0FD
:1022F000ECE7F1E10C947A2FFC016280448081E0EC
:102300008483E3E6F3E07490E2EEF3E0E491C091BD
:102310006D03C695C158D0E0CC0FDD1FCD2FDD2752
:10232000812C75E0972EAA24AA94B12C55245A9496
:10233000E719EE2EF12C80915F01881638F00E948B
:10234000DE0BCDB7DEB7E0E10C94962FC82CD12C74
:1023500082E0861568F09C9CF0019D9CF00D112494
:10236000E65EFC4F80916B03808380916C038183D8
:10237000411023C09C9CF0019D9CF00D1124E65E51
:10238000FC4F1382128220915D01C601820F911DC4
:102390009C01220F331F280F391F26513D4F9C9C53
:1023A000F0019D9CF00D1124E65EFC4F428161819D
:1023B00080810E9456068394BECF9C9C80019D9C88
:1023C000100D1124065E1C4FF80183818823F1F063
:1023D00081508383859DC0011124648170E00E9437
:1023E000BB2FFB01FF27ED59FC4F8491E82FE71924
:1023F000E59DC0011124B7010E94BB2F80916D03A0
:10240000689FB0011124F8017283BDCF0E944B3048
:10241000B5010E94CF2F8C179D070CF0B4CFF2E0CE
:10242000F61598F40E944B30B5010E94CF2FF801A9
:1024300080830E944B3020916C032695622F70E0C0
:102440000E94CF2F280FF80121839C9CF0019D9CB6
:10245000F00D1124E65EFC4F128280916D03893CE1
:1024600058F088EC9C9CF0019D9CF00D1124E65ED8
:10247000FC4F8483838387CF8431A0F784E1F2CF3C
:1024800060916A03669570E04BE050E08DE491E066
:102490000E945B30892B19F481E08093E5020E9451
:1024A0008C0F9093DF028093DE028091E6028460BD
:1024B0008093E6020895CF92DF92EF92FF926B0134
:1024C0007C010E944706B701A60188E090E00E94C7
:1024D000A430FF90EF90DF90CF900895A3E0B0E09C
:1024E000E4E7F2E10C94812F082FD62EF42EC22EB1
:1024F00090916A0390FF3CC020916B03281308C0A1
:1025000080916C03861304C080916D03841729F0B9
:102510008091E60282608093E602E92FE695AE2F75
:10252000B0E0A654BE4F8C918093E4029E7F92301F
:1025300019F59E012F5F3F4F4F2D6D2D802F0E946B
:1025400056064B8169818A810E946B0E00936B0352
:10255000D0926C03F0926D03CC2051F060916A032D
:1025600070916B0380916C0390916D030E945B12DC
:102570002396E9E00C949D2F823019F4F0906D03BE
:10258000E5CF8630A1F1893091F18931F9F6E95131
:102590006E2F6170B62EE695F0E0E25BFC4F149171
:1025A000E12C60915F01E61618F00E94DE0BCECFA1
:1025B000E19EC001112470E00E94BB2F802FB1105A
:1025C00014C0860F20915D01622F6E0D7727771F53
:1025D0009B01220F331F260F371F26513D4F4F2DD2
:1025E0006D2D0E945606E394DCCF861BEBCF022FA5
:1025F000ADCFEAE6F3E0438121E1421B08F440E07D
:1026000021E0628181810E946E120895EAE6F3E082
:10261000438121E1420F08F44FEF21E06281818183
:102620000E946E120895EAE6F3E0628121E1621BE6
:1026300008F460E021E0438181810E946E120895D8
:10264000EAE6F3E0628121E1620F08F46FEF21E036
:10265000438181810E946E120895EAE6F3E0818150
:1026600021E04381628188500E946E120895EAE65B
:10267000F3E0818121E043816281885F0E946E12D4
:10268000089580916E03882319F0815080936E0322
:1026900060916A0370916B0380916C0390916D035C
:1026A0000E945B12089580916E03833018F48F5F4F
:1026B00080936E0360916A0370916B0380916C0349
:1026C00090916D030E945B12089590916A0390FFB0
:1026D00031C0917081112FC0926090936A038091F4
:1026E000E60281608093E602662351F060916A03FE
:1026F00070916B0380916C0390916D030E945B124B
:1027000060916A03669570E04BE050E08DE491E0E3
:102710000E945B30892BB1F00E94400681E08093DB
:10272000E10220E040916D0360916C0380916B03A6
:102730000E946E1208958B3210F09465CECF880FF0
:10274000982BCBCF0E944012E9CF80916A038695E7
:10275000815009F48AE261E00E9465130895809136
:102760006A0386958F5F8B3208F081E061E00E94FA
:102770006513089590916A0390FF08C09695981785
:1027800028F0961718F40E94AF13089561E00E9494
:1027900065130895EAE6F3E087E1808311828FEF05
:1027A000828383831482A4EEB2E012968C911297F6
:1027B000836012968C9360817181828193810E94E3
:1027C0005B1208958091390290913802892B809391
:1027D000F60190913702992391F0892B8093F601AD
:1027E00020E088EF91E0FC013191CF0131112F5FA2
:1027F000F1E08E3F9F07B9F721111092370248E0B0
:1028000050E06FE272E086EF91E00E946830892B21
:10281000A9F088E0E6EFF1E0AFE2B2E001900D92BE
:102820008A95E1F7E0917103F0917203309731F0EE
:102830000280F381E02D86EF91E0099508958823C9
:1028400021F00E9471090E94E2130895882339F053
:1028500090913902982B909339020E94E2130895C7
:10286000882309F456C0823879F40E945E0F81FFF4
:1028700050C089E30E9485090E94E21389E30E9407
:1028800078090E94E2130895833859F40E945E0F7C
:1028900080FF3FC083E50E9485090E94E21383E523
:1028A000EECF843859F40E945E0F82FF32C087E475
:1028B0000E9485090E94E21387E4E1CF9CEF980F04
:1028C000913AE8F290E2980F983050F4877091E0D6
:1028D00001C0990F8A95EAF7892F0E947109D1CF1B
:1028E0009BE5980F933028F490E080E00E94FE056D
:1028F000089598E5980F9B3128F490E080E00E94BD
:10290000D905089593E3980F933118F460E00E947D
:10291000850A0895CF93C82F8823C9F08238C9F457
:102920000E945E0F81FD13C089E30E9485090E9409
:10293000E2132FEF87EE93E0215080409040E1F7C3
:1029400000C0000089E30E9478090E94E213CF9141
:1029500008958338A1F40E945E0F80FDF8CF83E5CF
:102960000E9485090E94E2132FEF81EE94E021502E
:1029700080409040E1F700C0000083E5E4CF843858
:10298000A1F40E945E0F82FDE2CF87E40E948509D8
:102990000E94E2132FEF81EE94E02150804090409E
:1029A000E1F700C0000087E4CECF8CEF8C0F813AB6
:1029B00068F4E8EFF1E08191C817E9F121E0EE3F1A
:1029C000F207C9F78C2F0E948509BFCF80E28C0FD8
:1029D000883068F4C77021E030E001C0220FCA954A
:1029E000EAF780913902822B80933902AECFEBE572
:1029F000EC0FE33040F4F0E0E159FE4F808190E0CD
:102A00000E94FE05A4CFE8E5EC0FEB3150F4F0E0B6
:102A1000EE0FFF1FEE58FE4F808191810E94D90575
:102A200096CF83E38C0F833108F091CF61E08C2F38
:102A30000E94850A8CCF8C2F0E9478090E94E21395
:102A4000C1CF1F93CF93DF93182FD0E0C0E089331D
:102A500011F4C0E5D0E0812F0E948A14209739F448
:102A6000812F0E943014DF91CF911F9108958FE93B
:102A70009FE00197F1F700C000002197EFCF0F937F
:102A80001F93CF93DF93C62FD42F022FFC01858194
:102A90008823A9F06093CD030E94CD059093CC03C9
:102AA0008093CB03C77081E001C0880FCA95EAF715
:102AB0000E942614DF91CF911F910F91089580916C
:102AC000CD03681332C08091CB039091CC030E9458
:102AD000B205883C910548F510E21D0FCD17B9F0FD
:102AE00080E28C0F883040F4C77081E001C0880F0D
:102AF000CA95EAF70E941F14183048F481E09D2F10
:102B0000977001C0880F9A95EAF70E942614802FCB
:102B10000E942115183070F6D77081E001C0880F2F
:102B2000DA95EAF70E941F14C5CFC77081E001C093
:102B3000880FCA95EAF7F6CF67EE7EEF90E080E067
:102B40000E94B03060E082E090E00E94923060E04D
:102B500083E090E00E94923010923A0260E074E1CB
:102B600084E090E00E94B03060E086E090E00E9457
:102B700092306FEF87E090E00E94923040E050E0AA
:102B8000BA0188E090E00E94A43060E08DE090E01F
:102B90000E94923040E050E0BA0188E190E00E944B
:102BA000A43060E087E190E00E94923040E050E085
:102BB000BA018CE190E00E94A43070E060E080E215
:102BC00090E00E94B03040E050E0BA0188E190E02F
:102BD0000E94A43080E00E944E100E94671040E0E6
:102BE00050E0BA018FE090E00E94A43040E050E055
:102BF000BA0183E190E00E94A430089590919A0276
:102C000092FB222720F9281779F080FB92F9909304
:102C10009A026091990270919A0284E090E00E9479
:102C2000B03082E00E945F0A089590E080E00E9448
:102C30008C30873E9E4F19F40E945D11089580E00C
:102C40000895CF9310923902C6E0E8EFF1E0DF017A
:102C50008C2F1D928A95E9F790E080E00E94FE0596
:102C600090E080E00E94D905109238020E94E213A1
:102C7000E8EDF2E0DF011D92CA95E9F71092D1026A
:102C80001092D2021092D3020E94EC06CF910895C6
:102C9000AAE2B0E0EEE4F6E10C94872F89E893E035
:102CA0002091F100DC012D93CD01B3E081399B0728
:102CB000B9F780918A03833009F472C0B8F4813087
:102CC00009F449C0823009F4B3C08091E80083FF61
:102CD0008BC28091890390918A039A3008F084C254
:102CE000E92FF0E0E55DFE4C0C94E32F8A3009F407
:102CF0008EC08B3009F471C0893039F78091890317
:102D0000813219F780918D0390918E03009711F015
:102D10000297D9F68091E800877F8093E800809140
:102D2000E80082FF38C09091F3008091F200029792
:102D300031F48091F100813011F0863021F48091DE
:102D4000F10080937C038091E8008B778093E8000A
:102D50000E94A504BACF80918903813A09F0B5CFCA
:102D60008091E800877F8093E80080918D039091A7
:102D70008E03892B61F468E08DE793E070E00E9498
:102D800051058091E8008B778093E8009ECF60E04A
:102D900090E080E0F3CF809187038111C0CF95CF81
:102DA00080918903813A09F090CF80918D039091B1
:102DB0008E03892B09F089CF8091E800877F80936B
:102DC000E8008091E80080FFFCCF80916001809353
:102DD000F1008091E8008E77B9CF8091890381322C
:102DE00009F073CF80918D0390918E03892B09F0A8
:102DF0006CCF8091E800877F8093E8000E94A50453
:102E000080918B03809360010E9421165ECF809198
:102E10008903813209F059CF8091E800877F809340
:102E2000E8000E94A50480918C0380937B034DCF22
:102E300080918903813A09F048CF8091E800877F2B
:102E40008093E8008091E80080FFFCCF80917B03B5
:102E5000BECF803899F0823809F0C6C180918D03C9
:102E60008F70873008F0C0C18093E9008091EB003B
:102E700085FB882780F91092E90006C080918503C0
:102E800090918603911182609091E800977F9093D2
:102E9000E8008093F1001092F1008091E8008E77B5
:102EA0009FC1882309F48DC1823009F09DC18091B2
:102EB0008B03811190C180918D038F702FEF280FAC
:102EC000263008F091C18093E9002091EB0020FFAB
:102ED00082C1933031F48091EB0080628093EB00EB
:102EE0007AC19091EB0090619093EB0021E030E08B
:102EF00001C0220F8A95EAF72093EA001092EA00B7
:102F00008091EB008860EACF81116EC110918B0334
:102F10001F778091E3008078812B8093E30080917C
:102F2000E800877F8093E8000E94A5048091E80074
:102F300080FFFCCF8091E30080688093E30082E013
:102F4000111183E0809387034FC18058823008F0CD
:102F50004BC120918B0330918C032C3DE3E03E0765
:102F6000A1F583E08A838AE289834FB7F894DE0172
:102F7000139620E03EE051E2E32FF0E0509357003B
:102F8000E49120FF03C0E295EF703F5FEF708E2F5A
:102F900090E0EA30C0F0C7968D939D932F5F243167
:102FA00059F74FBF8091E800877F8093E8006AE27D
:102FB00070E0CE0101960E9451058091E8008B7768
:102FC0008093E80011C1C096E7CF80918D03909166
:102FD0008E03432F55274330510509F44AC078F535
:102FE0004130510509F47AC08BE590E0E3E5F7E064
:102FF0004230510509F0F8C02091E800277F209366
:10300000E80020918F03309190038217930708F412
:103010009C0140E02115310509F065C0411163C0F4
:103020008091E80082FDC9CF80918703882329F22F
:10303000853019F28091E80083FFF2CFBECF413294
:10304000510509F43CC04232510509F0CDC083302E
:10305000910508F0C9C0FC01EE0FFF1FE851FE4FBB
:103060000190F081E02D8B519E4FDC018C9190E01E
:103070001AC0332721303105D1F02115310561F017
:103080002230310509F0B0C0E0ECF7E0E4918E2F7A
:1030900090E0E0ECF7E007C0E4EFF7E0E4918E2F7A
:1030A00090E0E4EFF7E0009709F49EC0A5CFE4EECE
:1030B000F7E0E4918E2F90E0E4EEF7E0F4CF833078
:1030C000910508F091C0880F991FFC01E251FE4F55
:1030D0000190F081E02D89E090E08ECF82E190E0D8
:1030E000EEEAF7E089CF80918703882309F465CF62
:1030F000853009F462CF8091E80083FD5ECF809136
:10310000E80082FD8DCF8091E80080FF83CF909111
:10311000F3008091F2002115310519F088309105F6
:1031200050F041E0089709F040E08091E8008E7788
:103130008093E8006FCF44914093F1003196215085
:1031400031090196E8CF803809F04EC08091E8003F
:10315000877F8093E800809188038093F1009DCE63
:10316000811142C010918B031230F0F58091E8007C
:10317000877F8093E800109388030E94A5041123A1
:1031800011F084E005C08091E30087FDFACF81E073
:103190008093870342E061EC81E00E94C40442E234
:1031A00061EC84E00E94C40442E261EC82E00E948F
:1031B000C40442E260EC83E00E94C404809187036F
:1031C00013C080918B03813079F481E0933009F052
:1031D00080E0809386031092E9008091E800877F69
:1031E0008093E8000E94A5048091E80083FF0AC054
:1031F0008091E800877F8093E8008091EB008062F7
:103200008093EB00AA96E3E00C94A32F0E94211672
:103210002FEF84E39CE0215080409040E1F700C014
:10322000000088E19CE00FB6F894A89580936000B8
:103230000FBE90936000FFCFA8E0B0E0E2E2F9E1BA
:103240000C947A2F8C01DC0114968C91882309F45C
:10325000CAC086E0F801DE01119601900D928A95B0
:10326000E1F7F801258189819A81222309F471C04F
:103270000E94FE10F82E682F89819A810E94150AFB
:1032800069817A818F2D0E94DF107C01D80115960B
:103290008C91882309F440C1C70197578038910564
:1032A00008F084C5BFE0BE1508F48DC08FEF93E031
:1032B0000E947E30811187C066E1A62E63E0B62EA3
:1032C000E1104BC0FE01339686E0DF011D928A9526
:1032D000E9F75AE0452E7501BFEFEB1AFB0AC5016D
:1032E0000E947E3089831A82882309F46CC0813061
:1032F00009F07DC06501E2E0CE0ED11CC7010E943D
:103300007E308A83882309F45EC09FEF980F933044
:1033100090F5F3E0AF0EB11CC6010E947E308B83A6
:10332000882309F450C01C82DE0111967D01F7014B
:103330002081222381F2213009F099C0918182817C
:10334000913009F056C0F2E0EF0EF11C0E942115F9
:1033500057C00E94CF09F82E93CFA114E4E0BE0617
:1033600091F1C5010E947E30811101C0EA94FFEF06
:10337000AF1ABF0AA5CF56018430B1F642E0E42E61
:10338000F12C56012FEFA21AB20AC6010E947E301C
:10339000E1E0F0E0EC0FFD1FEE0DFF1D80838823C0
:1033A00091F08C3741F4E2E0F0E0EC0FFD1FEE0D00
:1033B000FF1D1082B9CF3FEFE31AF30A650187E0E2
:1033C000E816F104F1F680912E02877061F0D801C1
:1033D00015968C91882339F080919A0282FF03C060
:1033E00082E00E945F0A2896E0E10C94962F570134
:1033F0009BCF923049F422E0E20EF11C0E948A1425
:10340000EFEFEE1AFE0A93CF933031F432E0E30E81
:10341000F11C0E943014F4CF943021F08FEFE81AA1
:10342000F80AEECF92E0E90EF11C30E020E0B7019F
:103430006F5F7F4FD70111964C918053990B8A3063
:10344000910550F021503109D8F2EFE9FFE03197B2
:10345000F1F700C00000F6CF429EF001439EF00D50
:1034600011249C012E0F3F1F842F7B01E0CFE22F00
:10347000F0E0E754FE4F5490822F8695869586950E
:1034800090E0FC01E755FE4F64902770712C022EEE
:1034900002C0759467940A94E2F731E063227724BE
:1034A000FC01E756FE4F8490912C022E02C09594A9
:1034B00087940A94E2F7A1E08A229924FC01E75755
:1034C000FE4FC490D12C02C0D594C7942A95E2F740
:1034D000B1E0CB22DD246114710419F081EE0E9469
:1034E0008A148114910419F086EE0E948A14852DA5
:1034F0000E9421158114910419F086EE0E94301467
:103500006114710419F081EE0E943014C114D104C9
:1035100009F476CF8CE21ACFF701E851FC47E73087
:10352000F10508F02FC4EB5CFE4C0C94E32F26E26F
:1035300041EE61EEC8010E943F1545CF27E245EEFE
:1035400065EEF8CF26E241EE60EEF4CF27E245EEDD
:1035500064EEF0CF26E241EE62EEECCF27E245EEDC
:1035600066EEE8CF28E241E0EBCF809199028160DE
:103570008093990295C080919A02886080939A0204
:103580008FC0809199028260F3CF8091990284600C
:10359000EFCF809199028860EBCF80919A02816091
:1035A000EDCF80919A028260E9CF8091990280618B
:1035B000DFCF809199028062DBCF80919902806495
:1035C000D7CF0E942116809199028068D1CF809137
:1035D00099028C60CDCF80919A028360CFCF809189
:1035E00099028E7FC5CF80919A02877FC7CF809145
:1035F00099028D7FBDCF809199028B7FB9CF809149
:103600009902877FB5CF80919A028E7FB7CF809144
:103610009A028D7FB3CF809199028F7EA9CF80913E
:1036200099028F7DA5CF809199028F7BA1CF0E94B7
:103630002116809199028F779BCF80919902837F89
:1036400097CF80919A028C7F99CF8091990282FBCB
:10365000992790F921E0922790FB82F990FB83F95A
:1036600087CF80919A02982F909591708E7F892BA9
:1036700090FB81F983CF90919902892F8F7B96FFE0
:10368000806476CF0E94211690919902892F97FB32
:1036900087F980586DCF61E08EE090E00E94923013
:1036A0006091990270919A0284E090E00E94B0309B
:1036B0000E94211688CE60E0EFCF90919902892F69
:1036C0008F7E94FF806154CF90919902892F8E7FD5
:1036D00090FF81604DCF90919A02892F877F93FF51
:1036E00088604CCF85E349C38091FE01811104C0FD
:1036F00089E20E94780943C385E3FBCFF7E7EF1621
:10370000FCE7FF0609F00CC381E00E94760A43E063
:1037100062E081E00E94320A56CE80916A0380FF07
:1037200017C08E7F80936A0360916A0370916B0368
:1037300080916C0390916D030E945B120E94400681
:103740008091E60281608093E6020E94DE0B3BCE10
:10375000816080936A0361E086950E94651333CE91
:1037600045EA53E16FEA73E10E9439062CCE4FEA35
:1037700053E165EA73E1F8CF4DE253E167E373E1AA
:10378000F3CF47E353E16DE273E1EECF43E153E161
:1037900060E273E1E9CF40E253E163E173E1E4CF3A
:1037A00049EF52E166E073E1DFCF46E053E169EFB4
:1037B00072E1DACF41E453E163E573E1D5CF43E54C
:1037C00053E161E473E1D0CF61E081E0C6CF65E011
:1037D00082E00E94BA13F7CD68E086E0FACF6EE08F
:1037E00089E0F7CF64E18FE0F4CF67E185E1F1CFC5
:1037F00061E088E1B2CF62E289E1EBCF61E083E290
:10380000ACCF6AE285E2E5CF27E7E2162CE7F206C5
:1038100009F457C038E7E3163CE7F30609F455C04E
:10382000F8018581E080F180882309F482C0C70116
:103830000E94FE10D82E682FC7010E94150AB701FA
:103840008D2D0E94DF100E9453087C01882ED80124
:103850001596AC90159716969C9092943FE0932203
:1038600080912E028770F1F0CA2CAA20E1F08F2DF2
:10387000807F803451F080E28E0D883098F0911076
:1038800004C08F2D807E803269F080919A0282FF81
:1038900009C082E00E945F0A80912E028770CC24CA
:1038A000C3948111C12CBF2CB2942FE0B222BBE093
:1038B000BB1508F4A5C0EB2DF0E0E45CFE4C0C94C5
:1038C000E32F81E00E94520A22CF82E0FBCFEBE59A
:1038D000EE16ECE7FE0659F1FCE5EF16FCE7FF06F5
:1038E000E1F02AE5E2162CE7F20609F099CF81E033
:1038F0001BC00E9421163FEF84E39CE031508040C2
:103900009040E1F700C000000E94BA0B6FEF7FEF1C
:1039100090E080E00E94B0301DC280919A0282FB4C
:10392000882780F991E089270E94FE1579CF80E0F1
:10393000FBCFC7010E94CF09D82E81CFEF2DEF70AA
:10394000DE2E8F2D807F19F0D29490EFD922AA20FD
:10395000B9F0DD2069F080E28E0D883010F0811022
:1039600009C080913902D82AD09239020E94E2130C
:103970008E2D44C080913802D82AD0923802F6CFDA
:103980008E2D0E943014DD20D9F180E28E0D88301A
:1039900010F0811004C08D2D0E94710906C0D094D2
:1039A00080913802D822D09238020E94E21328C0B7
:1039B000FF2DFF70DF2E8F2D807F803219F0D29483
:1039C00080EFD822882051F021E0821609F46DC0E2
:1039D000AA2009F479C09920E9F1CACF80919A020E
:1039E00082FD34C0AA2061F1DD2039F080913902D6
:1039F000D82AD09239020E94E21380E00E948A14F1
:103A0000AB2DA850BB0B149710F40E945E0FCC2076
:103A100009F4E9CC80912E0280FDE5CCF8011582F5
:103A20008695869586950E94760AC8010E941C1983
:103A300080912E028695869586950E94520AD3CC57
:103A400080E00E943014DD20D9F2A5CFAA2099F0A1
:103A5000911004C08D2D0E942614D2CF31E0931214
:103A6000CFCF809137029D2D9823D91649F2D82ABD
:103A7000D0923702C5CF9110C3CF8D2D0E941F1455
:103A8000909137028D2D892329F08D2D80958923E2
:103A9000809337028091FF019D2D982309F4B0CFC8
:103AA000D094D822D092FF01ABCFAA2029F085E094
:103AB000891508F4A5CFCECF94E0991508F4A0CFCE
:103AC0008D2D0E941F149CCF9920D1F3A9E38A1257
:103AD00009C0BFEFE7EEF3E0B150E040F040E1F79E
:103AE00000C000008E2D0E9430148ACF8F2D869545
:103AF0008695837061F0813009F082CFC7019370A1
:103B0000A11002C080E090E00E94D90579CFC701E2
:103B10009370A11002C080E090E00E94FE0570CF7B
:103B20006A2D8E2D0E94850A6BCF8F2D837091F5A3
:103B3000A11066CF4E2D429546954770440F440F15
:103B40008E2D8F70042E01C0880F0A94EAF72E2D57
:103B50002071E4FE07C02FE030E001C0220F4A953B
:103B6000EAF720953F2D369536953370323069F05F
:103B700050F440913A02313029F0822B84230E9484
:103B8000820A3ECF842B822BFACF282B80913A02D7
:103B90008227F5CF8695AA2011F08F2D817088237A
:103BA00009F42ECF4E2D429546954770440F440F91
:103BB0008E2D8F70042E01C0880F0A94EAF72E2DE7
:103BC0002071E4FE07C02FE030E001C0220F4A95CB
:103BD000EAF720953F2D369536953370323069F0EF
:103BE00050F440919802313029F0822B84230E94B6
:103BF0002F0A06CF842B822BFACF282B8091980294
:103C00008227F5CF2F2D2F70F22EAA2029F0822F98
:103C10000E94760A8E2D1FCF8E2D0E941F148F2D8D
:103C20000E94520AEDCE8E2D32EF8316B1F1381577
:103C300070F090EF8916D1F0A1EF8A1691F0AA20CA
:103C400009F45EC0911094CE8F2D8F712AC0B3EF0E
:103C50008B1651F1E4EF8E12F2CF80919A0282FD21
:103C60002FC08F2D8F71AA20D9F21BC0AA2081F0FE
:103C7000F4E0F91508F4C4CE2F2D2F7181E090E007
:103C800001C0880F2A95EAF7909198028927AFCF53
:103C900025E0291508F4B4CEEFCF8F2D8F71A11038
:103CA000BFCF0E94760AACCE80E0AA2009F49FCF55
:103CB0009F2D9F7181E001C0880F9A95EAF797CFF9
:103CC000AA2099F03F2D3F71F32E832F0E94760A90
:103CD00080919A0282FF07C0A8E0FA9EC0011124D9
:103CE000836080932E028F2DDCCF81E00E945F0ADB
:103CF000B1E0B91508F084CE82E00E945F0A80CE60
:103D0000992059F0893309F0EDCEEFEFF7EE23E07B
:103D1000E150F0402040E1F7E3CE8F2D8F7180CF4E
:103D200082E0F8E7EF16FCE7FF0609F4EECC83E04B
:103D3000E8168CE7F80609F4E9CD08F0C8CDE114DF
:103D4000ACE7FA0609F4D5CDB1E0EB16BCE7FB060B
:103D500009F066CD0E94061926E1E2162CE7F2066C
:103D600009F0CCCC809139028A7A91E009F490E094
:103D70009093FE018111B6CC89E20E9485090E94D0
:103D8000E21321CB36E1E3163CE7F30609F4ACCCB1
:103D9000809139028272F701E052F847E531F1056E
:103DA00008F032CDE85BFE4C0C94E32FF701E851AC
:103DB000FC47E730F10508F4B6CB1092CD03C701FC
:103DC0009057839748F684E090E00E948C3090935F
:103DD0009A0280939902F701E150F047E232F1052F
:103DE00008F0C3CBE35AFE4C0C94E32FCF93DF9340
:103DF00080912D02807F09F04DC080912C02882394
:103E000009F448C0E091CA0350919103C09128027F
:103E1000D09127026091290270912A0247E05E1733
:103E2000C9F18E2F90E0E49FF0011124EE56FC4F73
:103E30002481222391F1489FF001499FF00D112424
:103E4000DF01AE56BC4F11962C9111972C1325C053
:103E50002C912D1322C015962C91159721111DC060
:103E600012962D913C91261B370B283C3105A8F466
:103E700080912D028F70806180932D02E856FC4F57
